 earlyretbase

 Timestamp is 725a1e26 (reproducible build file hash)

 Preferred load address is 0000000180000000

 Start         Length     Name                   Class
 0001:00000000 00002f80H .text$mn                CODE
 0001:00002f80 00000036H .text$mn$00             CODE
 0001:00002fb6 00000092H .text$x                 CODE
 0002:00000000 00000198H .idata$5                DATA
 0002:00000198 00000038H .00cfg                  DATA
 0002:000001d0 00000008H .CRT$XCA                DATA
 0002:000001d8 00000008H .CRT$XCZ                DATA
 0002:000001e0 00000008H .CRT$XIA                DATA
 0002:000001e8 00000008H .CRT$XIC                DATA
 0002:000001f0 00000008H .CRT$XIZ                DATA
 0002:000001f8 00000008H .CRT$XLA                DATA
 0002:00000200 00000008H .CRT$XLZ                DATA
 0002:00000208 00000008H .CRT$XPA                DATA
 0002:00000210 00000008H .CRT$XPZ                DATA
 0002:00000218 00000008H .CRT$XTA                DATA
 0002:00000220 00000010H .CRT$XTZ                DATA
 0002:00000228 00000000H .gehcont$y              DATA
 0002:00000228 00000000H .gfids$y                DATA
 0002:00000230 000020d0H .rdata                  DATA
 0002:00002300 00000000H .rdata$CastGuardVftablesA DATA
 0002:00002300 00000000H .rdata$CastGuardVftablesC DATA
 0002:00002300 00000028H .rdata$T                DATA
 0002:00002328 000000b0H .rdata$voltmd           DATA
 0002:000023d8 00000320H .rdata$zzzdbg           DATA
 0002:000026f8 00000008H .rtc$IAA                DATA
 0002:00002700 00000008H .rtc$IZZ                DATA
 0002:00002708 00000008H .rtc$TAA                DATA
 0002:00002710 00000008H .rtc$TZZ                DATA
 0002:00002718 00000004H .tls                    DATA
 0002:0000271c 00000004H .tls$                   DATA
 0002:00002720 00000008H .tls$ZZZ                DATA
 0002:00002728 000002e8H .xdata                  DATA
 0002:00002a10 00000484H .edata                  DATA
 0002:00002e94 00000064H .idata$2                DATA
 0002:00002ef8 00000018H .idata$3                DATA
 0002:00002f10 00000198H .idata$4                DATA
 0002:000030a8 0000041cH .idata$6                DATA
 0003:00000000 00000090H .data                   DATA
 0003:00000090 0001b398H .bss                    DATA
 0004:00000000 000003b4H .pdata                  DATA

  Address         Publics by Value              Rva+Base               Lib:Object

 0000:00000000       __AbsoluteZero             0000000000000000     <absolute>
 0000:00000000       ___safe_se_handler_count   0000000000000000     <absolute>
 0000:00000000       ___safe_se_handler_table   0000000000000000     <absolute>
 0000:00000000       __arm64x_extra_rfe_table   0000000000000000     <absolute>
 0000:00000000       __arm64x_extra_rfe_table_size 0000000000000000     <absolute>
 0000:00000000       __arm64x_native_entrypoint 0000000000000000     <absolute>
 0000:00000000       __arm64x_redirection_metadata 0000000000000000     <absolute>
 0000:00000000       __arm64x_redirection_metadata_count 0000000000000000     <absolute>
 0000:00000000       __dynamic_value_reloc_table 0000000000000000     <absolute>
 0000:00000000       __enclave_config           0000000000000000     <absolute>
 0000:00000000       __guard_check_icall_a64n_fptr 0000000000000000     <absolute>
 0000:00000000       __guard_eh_cont_count      0000000000000000     <absolute>
 0000:00000000       __guard_eh_cont_table      0000000000000000     <absolute>
 0000:00000000       __guard_fids_count         0000000000000000     <absolute>
 0000:00000000       __guard_fids_table         0000000000000000     <absolute>
 0000:00000000       __guard_iat_count          0000000000000000     <absolute>
 0000:00000000       __guard_iat_table          0000000000000000     <absolute>
 0000:00000000       __guard_longjmp_count      0000000000000000     <absolute>
 0000:00000000       __guard_longjmp_table      0000000000000000     <absolute>
 0000:00000000       __hybrid_auxiliary_iat     0000000000000000     <absolute>
 0000:00000000       __hybrid_auxiliary_iat_copy 0000000000000000     <absolute>
 0000:00000000       __hybrid_code_map          0000000000000000     <absolute>
 0000:00000000       __hybrid_code_map_count    0000000000000000     <absolute>
 0000:00000000       __x64_code_ranges_to_entry_points 0000000000000000     <absolute>
 0000:00000000       __x64_code_ranges_to_entry_points_count 0000000000000000     <absolute>
 0000:00000100       __guard_flags              0000000000000100     <absolute>
 0000:00000000       __ImageBase                0000000180000000     <linker-defined>
 0001:00000000       ?NewObject@JNIEnv_@@QEAAPEAV_jobject@@PEAV_jclass@@PEAU_jmethodID@@ZZ 0000000180001000 f i libearlyretbase.obj
 0001:00000024       ?SetEventNotificationMode@_jvmtiEnv@@QEAA?AW4jvmtiError@@W4jvmtiEventMode@@W4jvmtiEvent@@PEAV_jobject@@ZZ 0000000180001024 f i libearlyretbase.obj
 0001:0000002c       ?TranslateError@@YAPEBDW4jvmtiError@@@Z 000000018000102c f   libearlyretbase.obj
 0001:000002e4       ?nsk_jni_check_exception@@YAHPEAUJNIEnv_@@QEBDH@Z 00000001800012e4 f   libearlyretbase.obj
 0001:00000428       ?nsk_jni_lverify@@YAHHPEAUJNIEnv_@@HQEBDH1ZZ 0000000180001428 f   libearlyretbase.obj
 0001:000004c8       Agent_Initialize           00000001800014c8 f   libearlyretbase.obj
 0001:00000638       Agent_OnAttach             0000000180001638 f   libearlyretbase.obj
 0001:00000638       Agent_OnLoad               0000000180001638 f   libearlyretbase.obj
 0001:00000640       FramePop                   0000000180001640 f   libearlyretbase.obj
 0001:0000066c       Java_nsk_jvmti_unit_FollowReferences_FollowRefObjects_addRefToVerify 000000018000166c f   libearlyretbase.obj
 0001:00000828       Java_nsk_jvmti_unit_FollowReferences_FollowRefObjects_getTag 0000000180001828 f   libearlyretbase.obj
 0001:000008e4       Java_nsk_jvmti_unit_FollowReferences_FollowRefObjects_resetRefsToVerify 00000001800018e4 f   libearlyretbase.obj
 0001:000008ec       Java_nsk_jvmti_unit_FollowReferences_FollowRefObjects_resetTags 00000001800018ec f   libearlyretbase.obj
 0001:00000930       Java_nsk_jvmti_unit_FollowReferences_FollowRefObjects_setTag 0000000180001930 f   libearlyretbase.obj
 0001:00000b7c       Java_nsk_jvmti_unit_ForceEarlyReturn_earlyretbase_check 0000000180001b7c f   libearlyretbase.obj
 0001:00000c08       Java_nsk_jvmti_unit_ForceEarlyReturn_earlyretbase_doForceEarlyReturn 0000000180001c08 f   libearlyretbase.obj
 0001:00000d7c       Java_nsk_jvmti_unit_ForceEarlyReturn_earlyretbase_resThread 0000000180001d7c f   libearlyretbase.obj
 0001:00000e00       Java_nsk_jvmti_unit_ForceEarlyReturn_earlyretbase_suspThread 0000000180001e00 f   libearlyretbase.obj
 0001:00000ed8       Java_nsk_share_jvmti_ArgumentHandler_getAgentOptionsString 0000000180001ed8 f   libearlyretbase.obj
 0001:00000f84       Java_nsk_share_jvmti_DebugeeClass_checkStatus 0000000180001f84 f   libearlyretbase.obj
 0001:0000100c       Java_nsk_share_jvmti_DebugeeClass_resetAgentData 000000018000200c f   libearlyretbase.obj
 0001:0000106c       Java_nsk_share_jvmti_RedefineAgent_agentStatus 000000018000206c f   libearlyretbase.obj
 0001:00001078       Java_nsk_share_jvmti_RedefineAgent_isRedefined 0000000180002078 f   libearlyretbase.obj
 0001:00001084       Java_nsk_share_jvmti_RedefineAgent_redefineAttempted 0000000180002084 f   libearlyretbase.obj
 0001:00001090       MA_checkStatus             0000000180002090 f   libearlyretbase.obj
 0001:00001134       MethodExit                 0000000180002134 f   libearlyretbase.obj
 0001:00001160       __local_stdio_printf_options 0000000180002160 f i libearlyretbase.obj
 0001:00001330       exitOnError                0000000180002330 f   libearlyretbase.obj
 0001:000013e4       fprintf                    00000001800023e4 f i libearlyretbase.obj
 0001:00001428       nsk_jvmti_lverify          0000000180002428 f   libearlyretbase.obj
 0001:00001518       nsk_jvmti_resetAgentData   0000000180002518 f   libearlyretbase.obj
 0001:0000158c       nsk_lcomplain              000000018000258c f   libearlyretbase.obj
 0001:000015ac       nsk_ldisplay               00000001800025ac f   libearlyretbase.obj
 0001:000015cc       nsk_ltrace                 00000001800025cc f   libearlyretbase.obj
 0001:000015ec       nsk_lvcomplain             00000001800025ec f   libearlyretbase.obj
 0001:000017a4       nsk_lvdisplay              00000001800027a4 f   libearlyretbase.obj
 0001:000017f0       nsk_lverify                00000001800027f0 f   libearlyretbase.obj
 0001:0000184c       nsk_lvtrace                000000018000284c f   libearlyretbase.obj
 0001:000018ac       nsk_printf                 00000001800028ac f   libearlyretbase.obj
 0001:000018d4       nsk_vprintf                00000001800028d4 f   libearlyretbase.obj
 0001:00001988       printf                     0000000180002988 f i libearlyretbase.obj
 0001:00001d08       suspendThreadAtMethod      0000000180002d08 f   libearlyretbase.obj
 0001:0000205c       __raise_securityfailure    000000018000305c f   MSVCRT:gs_report.obj
 0001:00002090       __report_gsfailure         0000000180003090 f   MSVCRT:gs_report.obj
 0001:000022d0       __GSHandlerCheck           00000001800032d0 f   MSVCRT:gshandler.obj
 0001:000022f0       __GSHandlerCheckCommon     00000001800032f0 f   MSVCRT:gshandler.obj
 0001:00002360       __security_check_cookie    0000000180003360 f   MSVCRT:amdsecgs.obj
 0001:000026a0       _DllMainCRTStartup         00000001800036a0 f   MSVCRT:dll_dllmain.obj
 0001:000026e0       __scrt_acquire_startup_lock 00000001800036e0 f   MSVCRT:utility.obj
 0001:0000271c       __scrt_dllmain_after_initialize_c 000000018000371c f   MSVCRT:utility.obj
 0001:00002750       __scrt_dllmain_before_initialize_c 0000000180003750 f   MSVCRT:utility.obj
 0001:00002768       __scrt_dllmain_crt_thread_attach 0000000180003768 f   MSVCRT:utility.obj
 0001:00002790       __scrt_dllmain_crt_thread_detach 0000000180003790 f   MSVCRT:utility.obj
 0001:000027a8       __scrt_dllmain_exception_filter 00000001800037a8 f   MSVCRT:utility.obj
 0001:00002808       __scrt_dllmain_uninitialize_c 0000000180003808 f   MSVCRT:utility.obj
 0001:00002838       __scrt_dllmain_uninitialize_critical 0000000180003838 f   MSVCRT:utility.obj
 0001:0000284c       __scrt_initialize_crt      000000018000384c f   MSVCRT:utility.obj
 0001:00002898       __scrt_initialize_onexit_tables 0000000180003898 f   MSVCRT:utility.obj
 0001:00002924       __scrt_is_nonwritable_in_current_image 0000000180003924 f   MSVCRT:utility.obj
 0001:000029bc       __scrt_release_startup_lock 00000001800039bc f   MSVCRT:utility.obj
 0001:000029e0       __scrt_uninitialize_crt    00000001800039e0 f   MSVCRT:utility.obj
 0001:00002a0c       _onexit                    0000000180003a0c f   MSVCRT:utility.obj
 0001:00002a48       atexit                     0000000180003a48 f   MSVCRT:utility.obj
 0001:00002a60       __crt_debugger_hook        0000000180003a60 f   MSVCRT:utility_desktop.obj
 0001:00002a68       __scrt_fastfail            0000000180003a68 f   MSVCRT:utility_desktop.obj
 0001:00002bb4       _guard_check_icall_nop     0000000180003bb4 f i MSVCRT:guard_support.obj
 0001:00002bb8       __security_init_cookie     0000000180003bb8 f   MSVCRT:gs_support.obj
 0001:00002c64       DllMain                    0000000180003c64 f   MSVCRT:dll_dllmain_stub.obj
 0001:00002c88       ?__scrt_initialize_type_info@@YAXXZ 0000000180003c88 f   MSVCRT:tncleanup.obj
 0001:00002c98       ?__scrt_uninitialize_type_info@@YAXXZ 0000000180003c98 f   MSVCRT:tncleanup.obj
 0001:00002ca4       __local_stdio_scanf_options 0000000180003ca4 f i MSVCRT:default_local_stdio_options.obj
 0001:00002cac       __scrt_initialize_default_local_stdio_options 0000000180003cac f   MSVCRT:default_local_stdio_options.obj
 0001:00002cc8       __scrt_get_dyn_tls_init_callback 0000000180003cc8 f   MSVCRT:dyn_tls_init.obj
 0001:00002cd0       _RTC_Initialize            0000000180003cd0 f   MSVCRT:initsect.obj
 0001:00002d0c       _RTC_Terminate             0000000180003d0c f   MSVCRT:initsect.obj
 0001:00002d48       __isa_available_init       0000000180003d48 f   MSVCRT:cpu_disp.obj
 0001:00002ef4       _get_startup_argv_mode     0000000180003ef4 f   MSVCRT:argv_mode.obj
 0001:00002efc       __scrt_is_ucrt_dll_in_use  0000000180003efc f   MSVCRT:ucrt_detection.obj
 0001:00002f10       memcpy                     0000000180003f10 f   vcruntime:VCRUNTIME140.dll
 0001:00002f16       memset                     0000000180003f16 f   vcruntime:VCRUNTIME140.dll
 0001:00002f1c       strchr                     0000000180003f1c f   vcruntime:VCRUNTIME140.dll
 0001:00002f22       __C_specific_handler       0000000180003f22 f   vcruntime:VCRUNTIME140.dll
 0001:00002f28       __std_type_info_destroy_list 0000000180003f28 f   vcruntime:VCRUNTIME140.dll
 0001:00002f2e       strlen                     0000000180003f2e f   ucrt:api-ms-win-crt-string-l1-1-0.dll
 0001:00002f34       _initterm                  0000000180003f34 f   ucrt:api-ms-win-crt-runtime-l1-1-0.dll
 0001:00002f3a       _initterm_e                0000000180003f3a f   ucrt:api-ms-win-crt-runtime-l1-1-0.dll
 0001:00002f40       _seh_filter_dll            0000000180003f40 f   ucrt:api-ms-win-crt-runtime-l1-1-0.dll
 0001:00002f46       _configure_narrow_argv     0000000180003f46 f   ucrt:api-ms-win-crt-runtime-l1-1-0.dll
 0001:00002f4c       _initialize_narrow_environment 0000000180003f4c f   ucrt:api-ms-win-crt-runtime-l1-1-0.dll
 0001:00002f52       _initialize_onexit_table   0000000180003f52 f   ucrt:api-ms-win-crt-runtime-l1-1-0.dll
 0001:00002f58       _register_onexit_function  0000000180003f58 f   ucrt:api-ms-win-crt-runtime-l1-1-0.dll
 0001:00002f5e       _execute_onexit_table      0000000180003f5e f   ucrt:api-ms-win-crt-runtime-l1-1-0.dll
 0001:00002f64       _crt_atexit                0000000180003f64 f   ucrt:api-ms-win-crt-runtime-l1-1-0.dll
 0001:00002f6a       _cexit                     0000000180003f6a f   ucrt:api-ms-win-crt-runtime-l1-1-0.dll
 0001:00002f70       __acrt_initialize          0000000180003f70 f   MSVCRT:ucrt_stubs.obj
 0001:00002f70       __acrt_thread_attach       0000000180003f70 f   MSVCRT:ucrt_stubs.obj
 0001:00002f70       __acrt_thread_detach       0000000180003f70 f   MSVCRT:ucrt_stubs.obj
 0001:00002f70       __acrt_uninitialize        0000000180003f70 f   MSVCRT:ucrt_stubs.obj
 0001:00002f70       __acrt_uninitialize_critical 0000000180003f70 f   MSVCRT:ucrt_stubs.obj
 0001:00002f70       __scrt_stub_for_acrt_initialize 0000000180003f70 f   MSVCRT:ucrt_stubs.obj
 0001:00002f70       __scrt_stub_for_acrt_thread_attach 0000000180003f70 f   MSVCRT:ucrt_stubs.obj
 0001:00002f70       __scrt_stub_for_acrt_thread_detach 0000000180003f70 f   MSVCRT:ucrt_stubs.obj
 0001:00002f70       __scrt_stub_for_acrt_uninitialize 0000000180003f70 f   MSVCRT:ucrt_stubs.obj
 0001:00002f70       __scrt_stub_for_acrt_uninitialize_critical 0000000180003f70 f   MSVCRT:ucrt_stubs.obj
 0001:00002f70       __vcrt_initialize          0000000180003f70 f   MSVCRT:ucrt_stubs.obj
 0001:00002f70       __vcrt_thread_attach       0000000180003f70 f   MSVCRT:ucrt_stubs.obj
 0001:00002f70       __vcrt_thread_detach       0000000180003f70 f   MSVCRT:ucrt_stubs.obj
 0001:00002f70       __vcrt_uninitialize        0000000180003f70 f   MSVCRT:ucrt_stubs.obj
 0001:00002f70       __vcrt_uninitialize_critical 0000000180003f70 f   MSVCRT:ucrt_stubs.obj
 0001:00002f74       __scrt_stub_for_is_c_termination_complete 0000000180003f74 f   MSVCRT:ucrt_stubs.obj
 0001:00002f74       _is_c_termination_complete 0000000180003f74 f   MSVCRT:ucrt_stubs.obj
 0001:00002f90       _guard_dispatch_icall_nop  0000000180003f90 f   MSVCRT:guard_dispatch.obj
 0001:00002fb0       _guard_xfg_dispatch_icall_nop 0000000180003fb0 f   MSVCRT:guard_xfg_dispatch.obj
 0002:00000000       __imp_Sleep                0000000180005000     kernel32:KERNEL32.dll
 0002:00000008       __imp_RtlCaptureContext    0000000180005008     kernel32:KERNEL32.dll
 0002:00000010       __imp_RtlLookupFunctionEntry 0000000180005010     kernel32:KERNEL32.dll
 0002:00000018       __imp_RtlVirtualUnwind     0000000180005018     kernel32:KERNEL32.dll
 0002:00000020       __imp_UnhandledExceptionFilter 0000000180005020     kernel32:KERNEL32.dll
 0002:00000028       __imp_SetUnhandledExceptionFilter 0000000180005028     kernel32:KERNEL32.dll
 0002:00000030       __imp_GetCurrentProcess    0000000180005030     kernel32:KERNEL32.dll
 0002:00000038       __imp_TerminateProcess     0000000180005038     kernel32:KERNEL32.dll
 0002:00000040       __imp_IsProcessorFeaturePresent 0000000180005040     kernel32:KERNEL32.dll
 0002:00000048       __imp_CloseHandle          0000000180005048     kernel32:KERNEL32.dll
 0002:00000050       __imp_InitializeCriticalSectionAndSpinCount 0000000180005050     kernel32:KERNEL32.dll
 0002:00000058       __imp_DeleteCriticalSection 0000000180005058     kernel32:KERNEL32.dll
 0002:00000060       __imp_CreateEventW         0000000180005060     kernel32:KERNEL32.dll
 0002:00000068       __imp_GetModuleHandleW     0000000180005068     kernel32:KERNEL32.dll
 0002:00000070       __imp_GetProcAddress       0000000180005070     kernel32:KERNEL32.dll
 0002:00000078       __imp_IsDebuggerPresent    0000000180005078     kernel32:KERNEL32.dll
 0002:00000080       __imp_QueryPerformanceCounter 0000000180005080     kernel32:KERNEL32.dll
 0002:00000088       __imp_GetCurrentProcessId  0000000180005088     kernel32:KERNEL32.dll
 0002:00000090       __imp_GetCurrentThreadId   0000000180005090     kernel32:KERNEL32.dll
 0002:00000098       __imp_GetSystemTimeAsFileTime 0000000180005098     kernel32:KERNEL32.dll
 0002:000000a0       __imp_DisableThreadLibraryCalls 00000001800050a0     kernel32:KERNEL32.dll
 0002:000000a8       __imp_InitializeSListHead  00000001800050a8     kernel32:KERNEL32.dll
 0002:000000b0       \177KERNEL32_NULL_THUNK_DATA 00000001800050b0     kernel32:KERNEL32.dll
 0002:000000b8       __imp_memcpy               00000001800050b8     vcruntime:VCRUNTIME140.dll
 0002:000000c0       __imp_memset               00000001800050c0     vcruntime:VCRUNTIME140.dll
 0002:000000c8       __imp_strchr               00000001800050c8     vcruntime:VCRUNTIME140.dll
 0002:000000d0       __imp___C_specific_handler 00000001800050d0     vcruntime:VCRUNTIME140.dll
 0002:000000d8       __imp___std_type_info_destroy_list 00000001800050d8     vcruntime:VCRUNTIME140.dll
 0002:000000e0       \177VCRUNTIME140_NULL_THUNK_DATA 00000001800050e0     vcruntime:VCRUNTIME140.dll
 0002:000000e8       __imp__errno               00000001800050e8     ucrt:api-ms-win-crt-runtime-l1-1-0.dll
 0002:000000f0       __imp_exit                 00000001800050f0     ucrt:api-ms-win-crt-runtime-l1-1-0.dll
 0002:000000f8       __imp__cexit               00000001800050f8     ucrt:api-ms-win-crt-runtime-l1-1-0.dll
 0002:00000100       __imp__crt_atexit          0000000180005100     ucrt:api-ms-win-crt-runtime-l1-1-0.dll
 0002:00000108       __imp__execute_onexit_table 0000000180005108     ucrt:api-ms-win-crt-runtime-l1-1-0.dll
 0002:00000110       __imp__register_onexit_function 0000000180005110     ucrt:api-ms-win-crt-runtime-l1-1-0.dll
 0002:00000118       __imp__initialize_onexit_table 0000000180005118     ucrt:api-ms-win-crt-runtime-l1-1-0.dll
 0002:00000120       __imp__initialize_narrow_environment 0000000180005120     ucrt:api-ms-win-crt-runtime-l1-1-0.dll
 0002:00000128       __imp__configure_narrow_argv 0000000180005128     ucrt:api-ms-win-crt-runtime-l1-1-0.dll
 0002:00000130       __imp__seh_filter_dll      0000000180005130     ucrt:api-ms-win-crt-runtime-l1-1-0.dll
 0002:00000138       __imp__initterm_e          0000000180005138     ucrt:api-ms-win-crt-runtime-l1-1-0.dll
 0002:00000140       __imp__initterm            0000000180005140     ucrt:api-ms-win-crt-runtime-l1-1-0.dll
 0002:00000148       \177api-ms-win-crt-runtime-l1-1-0_NULL_THUNK_DATA 0000000180005148     ucrt:api-ms-win-crt-runtime-l1-1-0.dll
 0002:00000150       __imp___acrt_iob_func      0000000180005150     ucrt:api-ms-win-crt-stdio-l1-1-0.dll
 0002:00000158       __imp_fflush               0000000180005158     ucrt:api-ms-win-crt-stdio-l1-1-0.dll
 0002:00000160       __imp___stdio_common_vsprintf 0000000180005160     ucrt:api-ms-win-crt-stdio-l1-1-0.dll
 0002:00000168       __imp___stdio_common_vfprintf 0000000180005168     ucrt:api-ms-win-crt-stdio-l1-1-0.dll
 0002:00000170       \177api-ms-win-crt-stdio-l1-1-0_NULL_THUNK_DATA 0000000180005170     ucrt:api-ms-win-crt-stdio-l1-1-0.dll
 0002:00000178       __imp__strdup              0000000180005178     ucrt:api-ms-win-crt-string-l1-1-0.dll
 0002:00000178       __imp_strdup               0000000180005178     ucrt:api-ms-win-crt-string-l1-1-0.dll
 0002:00000180       __imp_strlen               0000000180005180     ucrt:api-ms-win-crt-string-l1-1-0.dll
 0002:00000188       __imp_strncpy              0000000180005188     ucrt:api-ms-win-crt-string-l1-1-0.dll
 0002:00000190       \177api-ms-win-crt-string-l1-1-0_NULL_THUNK_DATA 0000000180005190     ucrt:api-ms-win-crt-string-l1-1-0.dll
 0002:00000198       __guard_check_icall_fptr   0000000180005198     MSVCRT:guard_support.obj
 0002:000001a0       __guard_xfg_check_icall_fptr 00000001800051a0     MSVCRT:guard_support.obj
 0002:000001a8       __guard_dispatch_icall_fptr 00000001800051a8     MSVCRT:guard_support.obj
 0002:000001b0       __guard_xfg_dispatch_icall_fptr 00000001800051b0     MSVCRT:guard_support.obj
 0002:000001b8       __guard_xfg_table_dispatch_icall_fptr 00000001800051b8     MSVCRT:guard_support.obj
 0002:000001c0       __castguard_check_failure_os_handled_fptr 00000001800051c0     MSVCRT:guard_support.obj
 0002:000001c8       __guard_memcpy_fptr        00000001800051c8     vcruntime:softmemtag.obj
 0002:000001d0       __xc_a                     00000001800051d0     MSVCRT:initializers.obj
 0002:000001d8       __xc_z                     00000001800051d8     MSVCRT:initializers.obj
 0002:000001e0       __xi_a                     00000001800051e0     MSVCRT:initializers.obj
 0002:000001f0       __xi_z                     00000001800051f0     MSVCRT:initializers.obj
 0002:000001f8       __xl_a                     00000001800051f8     MSVCRT:tlssup.obj
 0002:00000200       __xl_z                     0000000180005200     MSVCRT:tlssup.obj
 0002:00000208       __xp_a                     0000000180005208     MSVCRT:initializers.obj
 0002:00000210       __xp_z                     0000000180005210     MSVCRT:initializers.obj
 0002:00000218       __xt_a                     0000000180005218     MSVCRT:initializers.obj
 0002:00000220       __xt_z                     0000000180005220     MSVCRT:initializers.obj
 0002:00000230       g_refKindStr               0000000180005230     libearlyretbase.obj
 0002:000003e0       ??_C@_09BPLDFGCI@unknown_0@ 00000001800053e0     libearlyretbase.obj
 0002:000003f0       ??_C@_0BL@FPNMECJD@JVMTI_HEAP_REFERENCE_CLASS@ 00000001800053f0     libearlyretbase.obj
 0002:00000410       ??_C@_0BL@FKGKKLNM@JVMTI_HEAP_REFERENCE_FIELD@ 0000000180005410     libearlyretbase.obj
 0002:00000430       ??_C@_0CD@CAEHCFJF@JVMTI_HEAP_REFERENCE_ARRAY_ELEM@ 0000000180005430     libearlyretbase.obj
 0002:00000458       ??_C@_0CC@DNEBMCNK@JVMTI_HEAP_REFERENCE_CLASS_LOAD@ 0000000180005458     libearlyretbase.obj
 0002:00000480       ??_C@_0BN@CJMIPEBB@JVMTI_HEAP_REFERENCE_SIGNERS@ 0000000180005480     libearlyretbase.obj
 0002:000004a0       ??_C@_0CH@HBOIDPEB@JVMTI_HEAP_REFERENCE_PROTECTION@ 00000001800054a0     libearlyretbase.obj
 0002:000004c8       ??_C@_0BP@MDKGDGKL@JVMTI_HEAP_REFERENCE_INTERFACE@ 00000001800054c8     libearlyretbase.obj
 0002:000004e8       ??_C@_0CC@JJMIHNJH@JVMTI_HEAP_REFERENCE_STATIC_FIE@ 00000001800054e8     libearlyretbase.obj
 0002:00000510       ??_C@_0CD@IDHEEGID@JVMTI_HEAP_REFERENCE_CONSTANT_P@ 0000000180005510     libearlyretbase.obj
 0002:00000538       ??_C@_0CA@EFFCHNG@JVMTI_HEAP_REFERENCE_SUPERCLASS@ 0000000180005538     libearlyretbase.obj
 0002:00000558       ??_C@_0L@PCDFHGCJ@unknown_11@ 0000000180005558     libearlyretbase.obj
 0002:00000568       ??_C@_0L@NJBICFOK@unknown_12@ 0000000180005568     libearlyretbase.obj
 0002:00000578       ??_C@_0L@MAADBEKL@unknown_13@ 0000000180005578     libearlyretbase.obj
 0002:00000588       ??_C@_0L@IPECICGM@unknown_14@ 0000000180005588     libearlyretbase.obj
 0002:00000598       ??_C@_0L@JGFJLDCN@unknown_15@ 0000000180005598     libearlyretbase.obj
 0002:000005a8       ??_C@_0L@LNHEOAOO@unknown_16@ 00000001800055a8     libearlyretbase.obj
 0002:000005b8       ??_C@_0L@KEGPNBKP@unknown_17@ 00000001800055b8     libearlyretbase.obj
 0002:000005c8       ??_C@_0L@CDPHMNGA@unknown_18@ 00000001800055c8     libearlyretbase.obj
 0002:000005d8       ??_C@_0L@DKOMPMCB@unknown_19@ 00000001800055d8     libearlyretbase.obj
 0002:000005e8       ??_C@_0L@OJGIPJDB@unknown_20@ 00000001800055e8     libearlyretbase.obj
 0002:000005f8       ??_C@_0CA@KAOFNDEM@JVMTI_HEAP_REFERENCE_JNI_GLOBAL@ 00000001800055f8     libearlyretbase.obj
 0002:00000618       ??_C@_0CC@HPFAJBK@JVMTI_HEAP_REFERENCE_SYSTEM_CLA@ 0000000180005618     libearlyretbase.obj
 0002:00000640       ??_C@_0BN@FDEGFOHC@JVMTI_HEAP_REFERENCE_MONITOR@ 0000000180005640     libearlyretbase.obj
 0002:00000660       ??_C@_0CB@HKIBCMAJ@JVMTI_HEAP_REFERENCE_STACK_LOCA@ 0000000180005660     libearlyretbase.obj
 0002:00000688       ??_C@_0BP@EAACMMOE@JVMTI_HEAP_REFERENCE_JNI_LOCAL@ 0000000180005688     libearlyretbase.obj
 0002:000006a8       ??_C@_0BM@IJDEOGOE@JVMTI_HEAP_REFERENCE_THREAD@ 00000001800056a8     libearlyretbase.obj
 0002:000006c8       ??_C@_0BL@EDGPPKC@JVMTI_HEAP_REFERENCE_OTHER@ 00000001800056c8     libearlyretbase.obj
 0002:000006e4       ??_C@_04BCJPDBDA@Code@     00000001800056e4     libearlyretbase.obj
 0002:000006f0       ??_C@_0BA@OCLMCFKC@LineNumberTable@ 00000001800056f0     libearlyretbase.obj
 0002:00000700       ??_C@_0BD@CPAEPILC@LocalVariableTable@ 0000000180005700     libearlyretbase.obj
 0002:00000718       ??_C@_0BH@NMBDNHBD@LocalVariableTypeTable@ 0000000180005718     libearlyretbase.obj
 0002:00000730       ??_C@_0O@HIHEEDNJ@StackMapTable@ 0000000180005730     libearlyretbase.obj
 0002:00000740       ??_C@_03IGDHHNNC@?$CI?$CJJ@ 0000000180005740     libearlyretbase.obj
 0002:00000748       ??_C@_0N@MJKGCPBI@activeMethod@ 0000000180005748     libearlyretbase.obj
 0002:00000758       ??_C@_0L@HCDIAMJG@?9?5?$CFs?0?5?$CFd?3?5@ 0000000180005758     libearlyretbase.obj
 0002:00000770       ??_C@_0JI@HLPECLFI@?$CD?5?4?4?4?6?$CD?5ERROR?3?5too?5many?5complai@ 0000000180005770     libearlyretbase.obj
 0002:00000810       ??_C@_0ED@JNEKCCOB@The?5following?5fake?5exception?5st@ 0000000180005810     libearlyretbase.obj
 0002:00000858       ??_C@_0CN@FCNMDFBH@nsk?4share?4Fake_Exception_for_RU@ 0000000180005858     libearlyretbase.obj
 0002:00000888       ??_C@_08PGFFNAEI@?$CI?$CFs?3?$CFd?$CJ?5@ 0000000180005888     libearlyretbase.obj
 0002:00000898       ??_C@_0DP@IENMAEGI@s?2test?2hotspot?2jtreg?2vmTestbase@ 0000000180005898     libearlyretbase.obj
 0002:000008d8       ??_C@_0BL@NDJLFFJB@?7at?5nsk_lvcomplain?$CI?$CFs?3?$CFd?$CJ?6@ 00000001800058d8     libearlyretbase.obj
 0002:000008f8       ??_C@_0BC@JOOKAFKF@?$CD?5ERROR?3?5?$CFs?0?5?$CFd?3?5@ 00000001800058f8     libearlyretbase.obj
 0002:00000910       ??_C@_09KJEAHMEH@?$CD?5ERROR?3?5@ 0000000180005910     libearlyretbase.obj
 0002:0000091c       ??_C@_02GPIOPFAK@?$DO?$DO@ 000000018000591c     libearlyretbase.obj
 0002:00000920       ??_C@_02FODMEDOG@?$DM?$DM@ 0000000180005920     libearlyretbase.obj
 0002:00000924       ??_C@_02DJGKEECL@?4?4@     0000000180005924     libearlyretbase.obj
 0002:00000928       ??_C@_0O@CJPGJOAF@?9?5?$CFs?0?5?$CFd?3?5?$CFs?5@ 0000000180005928     libearlyretbase.obj
 0002:00000938       ??_C@_0CB@IAKPDOIC@?$CD?5?5?5verified?5assertion?5is?5FALSE@ 0000000180005938     libearlyretbase.obj
 0002:00000960       ??_C@_0CO@LGONDEPD@stdout?3?5fflush?5failed?5?9?5err?$DN?$CFd?5@ 0000000180005960     libearlyretbase.obj
 0002:00000990       ??_C@_0CO@KBGKJPBD@stderr?3?5fflush?5failed?5?9?5err?$DN?$CFd?5@ 0000000180005990     libearlyretbase.obj
 0002:000009c0       ??_C@_0BB@JCNMKLLK@JVMTI_ERROR_NONE@ 00000001800059c0     libearlyretbase.obj
 0002:000009d8       ??_C@_0BL@LDIMKLPH@JVMTI_ERROR_INVALID_THREAD@ 00000001800059d8     libearlyretbase.obj
 0002:000009f8       ??_C@_0CB@PJFPAIKJ@JVMTI_ERROR_INVALID_THREAD_GROU@ 00000001800059f8     libearlyretbase.obj
 0002:00000a20       ??_C@_0BN@LLMKHMNF@JVMTI_ERROR_INVALID_PRIORITY@ 0000000180005a20     libearlyretbase.obj
 0002:00000a40       ??_C@_0CB@MBOFKAGB@JVMTI_ERROR_THREAD_NOT_SUSPENDE@ 0000000180005a40     libearlyretbase.obj
 0002:00000a68       ??_C@_0BN@FABOLPBI@JVMTI_ERROR_THREAD_SUSPENDED@ 0000000180005a68     libearlyretbase.obj
 0002:00000a88       ??_C@_0BN@FDGNOBJM@JVMTI_ERROR_THREAD_NOT_ALIVE@ 0000000180005a88     libearlyretbase.obj
 0002:00000aa8       ??_C@_0BL@GOBIFKNJ@JVMTI_ERROR_INVALID_OBJECT@ 0000000180005aa8     libearlyretbase.obj
 0002:00000ac8       ??_C@_0BK@FCMAJPPC@JVMTI_ERROR_INVALID_CLASS@ 0000000180005ac8     libearlyretbase.obj
 0002:00000ae8       ??_C@_0BP@IKLLBKEB@JVMTI_ERROR_CLASS_NOT_PREPARED@ 0000000180005ae8     libearlyretbase.obj
 0002:00000b08       ??_C@_0BN@KLPPLKG@JVMTI_ERROR_INVALID_METHODID@ 0000000180005b08     libearlyretbase.obj
 0002:00000b28       ??_C@_0BN@BCEKOKND@JVMTI_ERROR_INVALID_LOCATION@ 0000000180005b28     libearlyretbase.obj
 0002:00000b48       ??_C@_0BM@DFDGPME@JVMTI_ERROR_INVALID_FIELDID@ 0000000180005b48     libearlyretbase.obj
 0002:00000b68       ??_C@_0BL@NELIEPEC@JVMTI_ERROR_NO_MORE_FRAMES@ 0000000180005b68     libearlyretbase.obj
 0002:00000b88       ??_C@_0BJ@BDBECFDM@JVMTI_ERROR_OPAQUE_FRAME@ 0000000180005b88     libearlyretbase.obj
 0002:00000ba8       ??_C@_0BK@MIIFNLOB@JVMTI_ERROR_TYPE_MISMATCH@ 0000000180005ba8     libearlyretbase.obj
 0002:00000bc8       ??_C@_0BJ@HPCAOILC@JVMTI_ERROR_INVALID_SLOT@ 0000000180005bc8     libearlyretbase.obj
 0002:00000be8       ??_C@_0BG@CHILOPNI@JVMTI_ERROR_DUPLICATE@ 0000000180005be8     libearlyretbase.obj
 0002:00000c00       ??_C@_0BG@DIEMLHKM@JVMTI_ERROR_NOT_FOUND@ 0000000180005c00     libearlyretbase.obj
 0002:00000c18       ??_C@_0BM@NHMCKHOB@JVMTI_ERROR_INVALID_MONITOR@ 0000000180005c18     libearlyretbase.obj
 0002:00000c38       ??_C@_0BO@PPEDAJGL@JVMTI_ERROR_NOT_MONITOR_OWNER@ 0000000180005c38     libearlyretbase.obj
 0002:00000c58       ??_C@_0BG@FCAIPEID@JVMTI_ERROR_INTERRUPT@ 0000000180005c58     libearlyretbase.obj
 0002:00000c70       ??_C@_0CB@EGDBNKOI@JVMTI_ERROR_INVALID_CLASS_FORMA@ 0000000180005c70     libearlyretbase.obj
 0002:00000c98       ??_C@_0CG@DGKOGIAL@JVMTI_ERROR_CIRCULAR_CLASS_DEFI@ 0000000180005c98     libearlyretbase.obj
 0002:00000cc0       ??_C@_0BP@ICEALPKC@JVMTI_ERROR_FAILS_VERIFICATION@ 0000000180005cc0     libearlyretbase.obj
 0002:00000ce0       ??_C@_0DC@JDACLMIO@JVMTI_ERROR_UNSUPPORTED_REDEFIN@ 0000000180005ce0     libearlyretbase.obj
 0002:00000d18       ??_C@_0DE@GKDKNOMJ@JVMTI_ERROR_UNSUPPORTED_REDEFIN@ 0000000180005d18     libearlyretbase.obj
 0002:00000d50       ??_C@_0BO@LAFKIOG@JVMTI_ERROR_INVALID_TYPESTATE@ 0000000180005d50     libearlyretbase.obj
 0002:00000d70       ??_C@_0DH@INDGCLLB@JVMTI_ERROR_UNSUPPORTED_REDEFIN@ 0000000180005d70     libearlyretbase.obj
 0002:00000da8       ??_C@_0DE@NHEOMMGI@JVMTI_ERROR_UNSUPPORTED_REDEFIN@ 0000000180005da8     libearlyretbase.obj
 0002:00000de0       ??_C@_0CA@EKPNJOEP@JVMTI_ERROR_UNSUPPORTED_VERSION@ 0000000180005de0     libearlyretbase.obj
 0002:00000e00       ??_C@_0BN@OFFMAHHL@JVMTI_ERROR_NAMES_DONT_MATCH@ 0000000180005e00     libearlyretbase.obj
 0002:00000e20       ??_C@_0DN@HHBBLAKE@JVMTI_ERROR_UNSUPPORTED_REDEFIN@ 0000000180005e20     libearlyretbase.obj
 0002:00000e60       ??_C@_0DO@HMBGBGNA@JVMTI_ERROR_UNSUPPORTED_REDEFIN@ 0000000180005e60     libearlyretbase.obj
 0002:00000ea0       ??_C@_0BP@PBECGKHJ@JVMTI_ERROR_UNMODIFIABLE_CLASS@ 0000000180005ea0     libearlyretbase.obj
 0002:00000ec0       ??_C@_0BK@CANILEHF@JVMTI_ERROR_NOT_AVAILABLE@ 0000000180005ec0     libearlyretbase.obj
 0002:00000ee0       ??_C@_0CE@INJKMEFK@JVMTI_ERROR_MUST_POSSESS_CAPABI@ 0000000180005ee0     libearlyretbase.obj
 0002:00000f08       ??_C@_0BJ@LBFPFPDM@JVMTI_ERROR_NULL_POINTER@ 0000000180005f08     libearlyretbase.obj
 0002:00000f28       ??_C@_0BP@CHJPNNEM@JVMTI_ERROR_ABSENT_INFORMATION@ 0000000180005f28     libearlyretbase.obj
 0002:00000f48       ??_C@_0BP@OMFMNLC@JVMTI_ERROR_INVALID_EVENT_TYPE@ 0000000180005f48     libearlyretbase.obj
 0002:00000f68       ??_C@_0BN@BIBNPHHO@JVMTI_ERROR_ILLEGAL_ARGUMENT@ 0000000180005f68     libearlyretbase.obj
 0002:00000f88       ??_C@_0BK@KKNDHDCE@JVMTI_ERROR_NATIVE_METHOD@ 0000000180005f88     libearlyretbase.obj
 0002:00000fa8       ??_C@_0BK@PMKCFHAE@JVMTI_ERROR_OUT_OF_MEMORY@ 0000000180005fa8     libearlyretbase.obj
 0002:00000fc8       ??_C@_0BK@NNJBDMNB@JVMTI_ERROR_ACCESS_DENIED@ 0000000180005fc8     libearlyretbase.obj
 0002:00000fe8       ??_C@_0BI@GHECLMNC@JVMTI_ERROR_WRONG_PHASE@ 0000000180005fe8     libearlyretbase.obj
 0002:00001000       ??_C@_0BF@OLIHJOII@JVMTI_ERROR_INTERNAL@ 0000000180006000     libearlyretbase.obj
 0002:00001018       ??_C@_0BO@EOHGKJHI@JVMTI_ERROR_UNATTACHED_THREAD@ 0000000180006018     libearlyretbase.obj
 0002:00001038       ??_C@_0CA@LKHFDACL@JVMTI_ERROR_INVALID_ENVIRONMENT@ 0000000180006038     libearlyretbase.obj
 0002:00001058       ??_C@_0BA@MMFHLOKK@?$DMunknown?5error?$DO@ 0000000180006058     libearlyretbase.obj
 0002:00001068       ??_C@_0CF@CBHOKDB@throwable?5?$DN?5jni?9?$DOExceptionOccur@ 0000000180006068     libearlyretbase.obj
 0002:00001090       ??_C@_03OFAPEBGM@?$CFs?6@  0000000180006090     libearlyretbase.obj
 0002:00001098       ??_C@_0DM@LPIGEGNJ@s?2test?2hotspot?2jtreg?2vmTestbase@ 0000000180006098     libearlyretbase.obj
 0002:000010d8       ??_C@_0CC@NFCNPEPK@Exception?5in?5JNI?5call?5?$CIcleared?$CJ@ 00000001800060d8     libearlyretbase.obj
 0002:00001100       ??_C@_0BJ@IBAKFIKF@jni?9?$DOExceptionDescribe?$CI?$CJ@ 0000000180006100     libearlyretbase.obj
 0002:00001120       ??_C@_0BG@GGKALKMH@jni?9?$DOExceptionClear?$CI?$CJ@ 0000000180006120     libearlyretbase.obj
 0002:00001138       ??_C@_0CF@JMGFGJLJ@?$CD?5?5?5verified?5JNI?5assertion?5is?5F@ 0000000180006138     libearlyretbase.obj
 0002:00001160       ??_C@_0CB@MLNJNCLJ@?5?5jvmti?5error?3?5code?$DN?$CFd?0?5name?$DN?$CFs@ 0000000180006160     libearlyretbase.obj
 0002:00001188       ??_C@_0CD@OHBGDKMK@?$CD?5?5?5jvmti?5error?3?5code?$DN?$CFd?0?5name?$DN@ 0000000180006188     libearlyretbase.obj
 0002:000011b0       ??_C@_0CG@JNNCGPHB@?$CD?5?5?5error?5expected?3?5code?$DN?$CFd?0?5na@ 00000001800061b0     libearlyretbase.obj
 0002:000011e0       ??_C@_0EB@IMGKPCGE@?$CIstr_obj?5?$DN?5jni?9?$DONewStringUTF?$CIco@ 00000001800061e0     libearlyretbase.obj
 0002:00001230       ??_C@_0EA@HFOGGBCC@s?2test?2hotspot?2jtreg?2vmTestbase@ 0000000180006230     libearlyretbase.obj
 0002:00001270       ??_C@_0CB@PKFNCBLK@?$DO?$DO?$DO?$DO?$DO?$DO?$DO?$DO?5Invoke?5SuspendThread?$CI?$CJ@ 0000000180006270     libearlyretbase.obj
 0002:00001298       ??_C@_0DC@FMKOEGFG@?$CFs?3?5Failed?5to?5call?5SuspendThrea@ 0000000180006298     libearlyretbase.obj
 0002:000012d0       ??_C@_0CO@HJKAMPK@?$CIGetFrameLocation?$CJ?5unexpected?5e@ 00000001800062d0     libearlyretbase.obj
 0002:00001300       ??_C@_0DJ@LJDGNGCH@?$DO?$DO?$DO?5Attempt?5?$CFd?5to?5suspend?5the?5t@ 0000000180006300     libearlyretbase.obj
 0002:00001340       ??_C@_0CK@GNODJBHO@?$CIResumeThread?$CJ?5unexpected?5error@ 0000000180006340     libearlyretbase.obj
 0002:00001370       ??_C@_0CL@KLNIBDFF@?$CISuspendThread?$CJ?5unexpected?5erro@ 0000000180006370     libearlyretbase.obj
 0002:000013a0       ??_C@_0CP@PCCFKDM@?$DM?$DM?$DM?$DM?$DM?$DM?$DM?$DM?5SuspendThread?$CI?$CJ?5is?5suc@ 00000001800063a0     libearlyretbase.obj
 0002:000013d0       ??_C@_0GE@PMCDEMIE@Failed?5in?5the?5suspendThread?3?5wa@ 00000001800063d0     libearlyretbase.obj
 0002:00001434       ??_C@_05KKCIMGE@error@     0000000180006434     libearlyretbase.obj
 0002:00001440       ??_C@_0EA@PNBCDMOA@s?2test?2hotspot?2jtreg?2vmTestbase@ 0000000180006440     libearlyretbase.obj
 0002:00001480       ??_C@_0DI@ILAHDLMP@?$CI?$CKagentThreadProc?$CJ?$CIjvmti_env?0?5a@ 0000000180006480     libearlyretbase.obj
 0002:000014b8       ??_C@_0BD@KDBALNLB@JVMTI?5agent?5thread@ 00000001800064b8     libearlyretbase.obj
 0002:000014d0       ??_C@_0BB@NOKBFPFO@java?1lang?1Thread@ 00000001800064d0     libearlyretbase.obj
 0002:000014e4       ??_C@_06FALKBLGB@?$DMinit?$DO@ 00000001800064e4     libearlyretbase.obj
 0002:000014f0       ??_C@_0BG@IKDDPPGD@?$CILjava?1lang?1String?$DL?$CJV@ 00000001800064f0     libearlyretbase.obj
 0002:00001510       ??_C@_0EB@IFJBFEKC@?$CIthreadClass?5?$DN?5jni_env?9?$DOFindCla@ 0000000180006510     libearlyretbase.obj
 0002:00001560       ??_C@_0GF@FGFIBKKL@?$CIthreadCtor?5?$DN?5jni_env?9?$DOGetMetho@ 0000000180006560     libearlyretbase.obj
 0002:000015c8       ??_C@_0DN@NCPDJLOG@?$CIthreadName?5?$DN?5jni_env?9?$DONewStrin@ 00000001800065c8     libearlyretbase.obj
 0002:00001610       ??_C@_0FE@PFKODBGC@?$CIthreadObject?5?$DN?5jni_env?9?$DONewObj@ 0000000180006610     libearlyretbase.obj
 0002:00001670       ??_C@_0ED@HOBAHHJI@?$CIthreadGlobalRef?5?$DN?5jni_env?9?$DONew@ 0000000180006670     libearlyretbase.obj
 0002:000016c0       ??_C@_0FN@HNJJAHFC@jvmti_env?9?$DORunAgentThread?$CIagent@ 00000001800066c0     libearlyretbase.obj
 0002:00001720       ??_C@_0EA@MOJDNKDF@Debuggee?5status?5sync?5aborted?5be@ 0000000180006720     libearlyretbase.obj
 0002:00001760       ??_C@_0EA@EEOEJAEN@status?5?$DN?5syncDebuggeeStatus?$CIjni@ 0000000180006760     libearlyretbase.obj
 0002:000017a0       ??_C@_0BL@JBCFNBMB@nsk_jvmti_resetAgentData?$CI?$CJ@ 00000001800067a0     libearlyretbase.obj
 0002:000017c0       ??_C@_0EL@LPBEELIP@s?2test?2hotspot?2jtreg?2vmTestbase@ 00000001800067c0     libearlyretbase.obj
 0002:00001810       ??_C@_0CK@JDAMFDMJ@jvmti?9?$DOSetTag?$CIo?0?5tag?$CJ?5?$DN?$DN?5JVMTI_@ 0000000180006810     libearlyretbase.obj
 0002:00001840       ??_C@_0CC@DAMNHKNI@Can?8t?5set?5tag?5?$CFli?5for?5object?5?$CFl@ 0000000180006840     libearlyretbase.obj
 0002:00001868       ??_C@_0DL@HAJPNKEF@jvmti?9?$DOGetObjectHashCode?$CIo?0?5?$CGha@ 0000000180006868     libearlyretbase.obj
 0002:000018a8       ??_C@_0BL@JFPIEOBF@Can?8t?5get?5hash?5object?5?$CFlx?6@ 00000001800068a8     libearlyretbase.obj
 0002:000018c8       ??_C@_0BG@DICPHBKN@setTag?3?5?$CF08x?5?$DM?9?5?$CF?53li@ 00000001800068c8     libearlyretbase.obj
 0002:000018e0       ??_C@_0DH@FCEEBDMJ@?$CIs?5?$DN?5jni?9?$DOGetStringUTFChars?$CIsIn@ 00000001800068e0     libearlyretbase.obj
 0002:00001918       ??_C@_0BJ@OKKGHDCN@Can?8t?5get?5string?5at?5?$CF?$CDp?6@ 0000000180006918     libearlyretbase.obj
 0002:00001938       ??_C@_0BP@EKFLGGFJ@Can?8t?5get?5string?5at?5?$CF?$CDp?3?5null?6@ 0000000180006938     libearlyretbase.obj
 0002:00001958       ??_C@_06ICODBHCL@?5?1?1?5?$CFs@ 0000000180006958     libearlyretbase.obj
 0002:00001960       ??_C@_0DB@KGFPLEGO@?$CIr?5?$DN?5jvmti?9?$DOGetTag?$CIo?0?5?$CGtag?$CJ?$CJ?5?$DN?$DN@ 0000000180006960     libearlyretbase.obj
 0002:00001998       ??_C@_0CO@PDAGBCGJ@Can?8t?5GetTag?5for?5object?5?$CFlx?4?5Re@ 0000000180006998     libearlyretbase.obj
 0002:000019c8       ??_C@_0CH@HPEODOHC@TEST_BUG?3?5Max?4?5number?5of?5refs?5r@ 00000001800069c8     libearlyretbase.obj
 0002:000019f0       ??_C@_0DI@PHFCABIM@?$CIr?5?$DN?5jvmti?9?$DOGetTag?$CIfrom?0?5?$CGtagFr@ 00000001800069f0     libearlyretbase.obj
 0002:00001a28       ??_C@_0DI@MDEGFNKD@TEST_BUG?3?5Can?8t?5GetTag?5for?5obje@ 0000000180006a28     libearlyretbase.obj
 0002:00001a60       ??_C@_0DE@MLELJAHM@?$CIr?5?$DN?5jvmti?9?$DOGetTag?$CIto?0?5?$CGtagTo?$CJ?$CJ@ 0000000180006a60     libearlyretbase.obj
 0002:00001a98       ??_C@_0CF@CKNHIJHL@?$CD?$CD?$CD?$CD?5MethodExit?5event?5occurred?5@ 0000000180006a98     libearlyretbase.obj
 0002:00001ac0       ??_C@_0CD@GAGNNEOH@?$CD?$CD?$CD?$CD?5FramePop?5event?5occurred?5?$CD?$CD@ 0000000180006ac0     libearlyretbase.obj
 0002:00001ae8       ??_C@_0CD@MAPGAMMD@Cannot?5get?5class?5of?5thread?5obje@ 0000000180006ae8     libearlyretbase.obj
 0002:00001b10       ??_C@_0CF@FPPLGJAO@Cannot?5find?5Method?5ID?5for?5metho@ 0000000180006b10     libearlyretbase.obj
 0002:00001b38       ??_C@_0CA@LCONHFJP@?$DO?$DO?$DO?$DO?$DO?$DO?$DO?$DO?5Invoke?5ResumeThread?$CI?$CJ?6@ 0000000180006b38     libearlyretbase.obj
 0002:00001b60       ??_C@_0FO@ELLGBMOH@s?2test?2hotspot?2jtreg?2vmTestbase@ 0000000180006b60     libearlyretbase.obj
 0002:00001bc0       ??_C@_0DB@GNNPBNHM@?$CFs?3?5Failed?5to?5call?5ResumeThread@ 0000000180006bc0     libearlyretbase.obj
 0002:00001bf8       ??_C@_0CO@ONBIKMHM@?$DM?$DM?$DM?$DM?$DM?$DM?$DM?$DM?5ResumeThread?$CI?$CJ?5is?5succ@ 0000000180006bf8     libearlyretbase.obj
 0002:00001c28       ??_C@_0CN@GHJIKGLO@Failed?5to?5enable?5METHOD_EXIT?5ev@ 0000000180006c28     libearlyretbase.obj
 0002:00001c58       ??_C@_0CL@EPIEADBE@Failed?5to?5enable?5FRAME_POP?5even@ 0000000180006c58     libearlyretbase.obj
 0002:00001c88       ??_C@_0CM@DJHCDKC@?$CINotifyFramePop?$CJ?5unexpected?5err@ 0000000180006c88     libearlyretbase.obj
 0002:00001cb8       ??_C@_0CE@PFFEPIEI@?$DO?$DO?$DO?$DO?$DO?$DO?$DO?$DO?5Invoke?5ForceEarlyRetur@ 0000000180006cb8     libearlyretbase.obj
 0002:00001ce0       ??_C@_0EI@NCHOHAEJ@TEST?5FAILED?3?5the?5function?5Force@ 0000000180006ce0     libearlyretbase.obj
 0002:00001d28       ??_C@_0DF@KIBMOCOK@?7For?5more?5info?5about?5this?5error@ 0000000180006d28     libearlyretbase.obj
 0002:00001d60       ??_C@_0DK@NJGINIAG@Check?5?$CD1?5PASSED?3?5ForceEarlyRetu@ 0000000180006d60     libearlyretbase.obj
 0002:00001da0       ??_C@_0CP@GHNALCAI@Wrong?5error?5code?5from?5a?5valid?5c@ 0000000180006da0     libearlyretbase.obj
 0002:00001dd0       ??_C@_0DG@LAJPGIIE@?$CIGetPotentialCapabilities?$CJ?5unex@ 0000000180006dd0     libearlyretbase.obj
 0002:00001e08       ??_C@_0CN@LKPEOJPO@?$CIAddCapabilities?$CJ?5unexpected?5er@ 0000000180006e08     libearlyretbase.obj
 0002:00001e38       ??_C@_0CN@BCCBOHCH@?$CIGetCapabilities?$CJ?5unexpected?5er@ 0000000180006e38     libearlyretbase.obj
 0002:00001e68       ??_C@_0CO@KFILKBDH@Warning?3?5ForceEarlyReturn?5is?5no@ 0000000180006e68     libearlyretbase.obj
 0002:00001e98       ??_C@_0CM@FEKJDMLD@Warning?3?5suspend?1resume?5is?5not?5@ 0000000180006e98     libearlyretbase.obj
 0002:00001ec8       ??_C@_0CP@IMINGNLL@?$CISetEventCallbacks?$CJ?5unexpected?5@ 0000000180006ec8     libearlyretbase.obj
 0002:00001ef8       ??_C@_0DK@CDIPDFNJ@Warning?3?5FramePop?5or?5MethodExit@ 0000000180006ef8     libearlyretbase.obj
 0002:00001f38       ??_C@_0DG@PDDENJIG@JVMTI?5?5PopFrame?5?5events?3?5expect@ 0000000180006f38     libearlyretbase.obj
 0002:00001f70       ??_C@_0DG@GKAGOOPB@JVMTI?5MethodExit?5events?3?5expect@ 0000000180006f70     libearlyretbase.obj
 0002:00001fb0       ??_C@_0EI@IHGGBMFG@TEST?5FAILED?3?5JVMTI?5MethodExit?5o@ 0000000180006fb0     libearlyretbase.obj
 0002:00002000       ??_C@_0EL@CHKEOCAG@Check?5?$CD2?5PASSED?3?5JVMTI?5MethodEx@ 0000000180007000     libearlyretbase.obj
 0002:00002060       ??_C@_1EC@JIJBPKFM@?$AAa?$AAp?$AAi?$AA?9?$AAm?$AAs?$AA?9?$AAw?$AAi?$AAn?$AA?9?$AAc?$AAo?$AAr?$AAe@ 0000000180007060     MSVCRT:thread_safe_statics.obj
 0002:000020a8       ??_C@_1BK@MGMFAEKH@?$AAk?$AAe?$AAr?$AAn?$AAe?$AAl?$AA3?$AA2?$AA?4?$AAd?$AAl?$AAl@ 00000001800070a8     MSVCRT:thread_safe_statics.obj
 0002:000020c8       ??_C@_0BJ@JEBJOJFJ@SleepConditionVariableCS@ 00000001800070c8     MSVCRT:thread_safe_statics.obj
 0002:000020e8       ??_C@_0BJ@PGPPEPCC@WakeAllConditionVariable@ 00000001800070e8     MSVCRT:thread_safe_statics.obj
 0002:00002108       _pDefaultRawDllMain        0000000180007108     MSVCRT:dll_dllmain.obj
 0002:00002108       _pRawDllMain               0000000180007108     MSVCRT:dll_dllmain.obj
 0002:00002110       __xmm@ffffffffffffffffffffffffffffffff 0000000180007110     MSVCRT:utility.obj
 0002:00002120       _load_config_used          0000000180007120     MSVCRT:loadcfg.obj
 0002:00002300       _tls_used                  0000000180007300     MSVCRT:tlssup.obj
 0002:00002328       __volatile_metadata        0000000180007328     <linker-defined>
 0002:000026f8       __rtc_iaa                  00000001800076f8     MSVCRT:initsect.obj
 0002:00002700       __rtc_izz                  0000000180007700     MSVCRT:initsect.obj
 0002:00002708       __rtc_taa                  0000000180007708     MSVCRT:initsect.obj
 0002:00002710       __rtc_tzz                  0000000180007710     MSVCRT:initsect.obj
 0002:00002718       _tls_start                 0000000180007718     MSVCRT:tlssup.obj
 0002:0000271c       _Init_thread_epoch         000000018000771c     MSVCRT:thread_safe_statics.obj
 0002:00002720       _tls_end                   0000000180007720     MSVCRT:tlssup.obj
 0002:00002e94       __IMPORT_DESCRIPTOR_KERNEL32 0000000180007e94     kernel32:KERNEL32.dll
 0002:00002ea8       __IMPORT_DESCRIPTOR_VCRUNTIME140 0000000180007ea8     vcruntime:VCRUNTIME140.dll
 0002:00002ebc       __IMPORT_DESCRIPTOR_api-ms-win-crt-runtime-l1-1-0 0000000180007ebc     ucrt:api-ms-win-crt-runtime-l1-1-0.dll
 0002:00002ed0       __IMPORT_DESCRIPTOR_api-ms-win-crt-stdio-l1-1-0 0000000180007ed0     ucrt:api-ms-win-crt-stdio-l1-1-0.dll
 0002:00002ee4       __IMPORT_DESCRIPTOR_api-ms-win-crt-string-l1-1-0 0000000180007ee4     ucrt:api-ms-win-crt-string-l1-1-0.dll
 0002:00002ef8       __NULL_IMPORT_DESCRIPTOR   0000000180007ef8     kernel32:KERNEL32.dll
 0003:00000040       _Init_global_epoch         0000000180009040     MSVCRT:thread_safe_statics.obj
 0003:00000050       __security_cookie          0000000180009050     MSVCRT:gs_cookie.obj
 0003:00000058       __security_cookie_complement 0000000180009058     MSVCRT:gs_cookie.obj
 0003:00000060       __scrt_native_dllmain_reason 0000000180009060     MSVCRT:utility.obj
 0003:00000068       __isa_available            0000000180009068     MSVCRT:cpu_disp.obj
 0003:0000006c       __isa_enabled              000000018000906c     MSVCRT:cpu_disp.obj
 0003:00000070       __memset_fast_string_threshold 0000000180009070     MSVCRT:cpu_disp.obj
 0003:00000078       __memset_nt_threshold      0000000180009078     MSVCRT:cpu_disp.obj
 0003:00000080       __scrt_ucrt_dll_is_in_use  0000000180009080     MSVCRT:ucrt_stubs.obj
 0003:00000090       g_wrongHeapCallbacks       0000000180009090     libearlyretbase.obj
 0003:00000110       g_szTagInfo                0000000180009110     libearlyretbase.obj
 0003:00002050       g_tagFlags                 000000018000b050     libearlyretbase.obj
 0003:00002438       g_refsToVerifyCnt          000000018000b438     libearlyretbase.obj
 0003:0000243c       g_fakeUserData             000000018000b43c     libearlyretbase.obj
 0003:00002440       g_tagVisitCount            000000018000b440     libearlyretbase.obj
 0003:000033e0       g_refsToVerify             000000018000c3e0     libearlyretbase.obj
 0003:0001aae0       g_userDataError            0000000180023ae0     libearlyretbase.obj
 0003:0001ade0       ?_OptionsStorage@?1??__local_stdio_printf_options@@9@4_KA 0000000180023de0     libearlyretbase.obj
 0003:0001b3a8       _tls_index                 00000001800243a8     MSVCRT:tlssup.obj
 0003:0001b3b0       __scrt_current_native_startup_state 00000001800243b0     MSVCRT:utility.obj
 0003:0001b3b8       __scrt_native_startup_lock 00000001800243b8     MSVCRT:utility.obj
 0003:0001b3f8       __scrt_debugger_hook_flag  00000001800243f8     MSVCRT:utility_desktop.obj
 0003:0001b400       ?__type_info_root_node@@3U__type_info_node@@A 0000000180024400     MSVCRT:tncleanup.obj
 0003:0001b410       ?_OptionsStorage@?1??__local_stdio_scanf_options@@9@4_KA 0000000180024410     MSVCRT:default_local_stdio_options.obj
 0003:0001b418       __favor                    0000000180024418     MSVCRT:cpu_disp.obj
 0003:0001b420       __dyn_tls_init_callback    0000000180024420     <common>

 entry point at        0001:000026a0

 Static symbols

 0000:fffd9000       .debug$S                   0000000180000000     earlyretbase.exp
 0000:fffd9000       .debug$S                   0000000180000000     vcruntime:VCRUNTIME140.dll
 0000:fffd9000       .debug$S                   0000000180000000     vcruntime:VCRUNTIME140.dll
 0000:fffd9000       .debug$S                   0000000180000000     vcruntime:VCRUNTIME140.dll
 0000:fffd9000       .debug$S                   0000000180000000     vcruntime:VCRUNTIME140.dll
 0000:fffd9000       .debug$S                   0000000180000000     vcruntime:VCRUNTIME140.dll
 0000:fffd9000       .debug$S                   0000000180000000     vcruntime:VCRUNTIME140.dll
 0000:fffd9000       .debug$S                   0000000180000000     vcruntime:VCRUNTIME140.dll
 0000:fffd9000       .debug$S                   0000000180000000     ucrt:api-ms-win-crt-convert-l1-1-0.dll
 0002:ffffb000       .idata$6                   0000000180000000     ucrt:api-ms-win-crt-convert-l1-1-0.dll
 0000:fffd9000       .debug$S                   0000000180000000     ucrt:api-ms-win-crt-heap-l1-1-0.dll
 0000:fffd9000       .debug$S                   0000000180000000     ucrt:api-ms-win-crt-heap-l1-1-0.dll
 0000:fffd9000       .debug$S                   0000000180000000     ucrt:api-ms-win-crt-heap-l1-1-0.dll
 0000:fffd9000       .debug$S                   0000000180000000     ucrt:api-ms-win-crt-heap-l1-1-0.dll
 0002:ffffb000       .idata$6                   0000000180000000     ucrt:api-ms-win-crt-heap-l1-1-0.dll
 0000:fffd9000       .debug$S                   0000000180000000     ucrt:api-ms-win-crt-runtime-l1-1-0.dll
 0000:fffd9000       .debug$S                   0000000180000000     ucrt:api-ms-win-crt-runtime-l1-1-0.dll
 0000:fffd9000       .debug$S                   0000000180000000     ucrt:api-ms-win-crt-runtime-l1-1-0.dll
 0000:fffd9000       .debug$S                   0000000180000000     ucrt:api-ms-win-crt-runtime-l1-1-0.dll
 0000:fffd9000       .debug$S                   0000000180000000     ucrt:api-ms-win-crt-runtime-l1-1-0.dll
 0000:fffd9000       .debug$S                   0000000180000000     ucrt:api-ms-win-crt-runtime-l1-1-0.dll
 0000:fffd9000       .debug$S                   0000000180000000     ucrt:api-ms-win-crt-runtime-l1-1-0.dll
 0000:fffd9000       .debug$S                   0000000180000000     ucrt:api-ms-win-crt-runtime-l1-1-0.dll
 0000:fffd9000       .debug$S                   0000000180000000     ucrt:api-ms-win-crt-runtime-l1-1-0.dll
 0000:fffd9000       .debug$S                   0000000180000000     ucrt:api-ms-win-crt-runtime-l1-1-0.dll
 0000:fffd9000       .debug$S                   0000000180000000     ucrt:api-ms-win-crt-runtime-l1-1-0.dll
 0000:fffd9000       .debug$S                   0000000180000000     ucrt:api-ms-win-crt-runtime-l1-1-0.dll
 0000:fffd9000       .debug$S                   0000000180000000     ucrt:api-ms-win-crt-runtime-l1-1-0.dll
 0000:fffd9000       .debug$S                   0000000180000000     ucrt:api-ms-win-crt-runtime-l1-1-0.dll
 0000:fffd9000       .debug$S                   0000000180000000     ucrt:api-ms-win-crt-runtime-l1-1-0.dll
 0000:fffd9000       .debug$S                   0000000180000000     ucrt:api-ms-win-crt-runtime-l1-1-0.dll
 0000:fffd9000       .debug$S                   0000000180000000     ucrt:api-ms-win-crt-stdio-l1-1-0.dll
 0000:fffd9000       .debug$S                   0000000180000000     ucrt:api-ms-win-crt-stdio-l1-1-0.dll
 0000:fffd9000       .debug$S                   0000000180000000     ucrt:api-ms-win-crt-stdio-l1-1-0.dll
 0000:fffd9000       .debug$S                   0000000180000000     ucrt:api-ms-win-crt-stdio-l1-1-0.dll
 0000:fffd9000       .debug$S                   0000000180000000     ucrt:api-ms-win-crt-stdio-l1-1-0.dll
 0000:fffd9000       .debug$S                   0000000180000000     ucrt:api-ms-win-crt-stdio-l1-1-0.dll
 0000:fffd9000       .debug$S                   0000000180000000     ucrt:api-ms-win-crt-stdio-l1-1-0.dll
 0000:fffd9000       .debug$S                   0000000180000000     ucrt:api-ms-win-crt-stdio-l1-1-0.dll
 0000:fffd9000       .debug$S                   0000000180000000     ucrt:api-ms-win-crt-stdio-l1-1-0.dll
 0000:fffd9000       .debug$S                   0000000180000000     ucrt:api-ms-win-crt-stdio-l1-1-0.dll
 0000:fffd9000       .debug$S                   0000000180000000     ucrt:api-ms-win-crt-string-l1-1-0.dll
 0000:fffd9000       .debug$S                   0000000180000000     ucrt:api-ms-win-crt-string-l1-1-0.dll
 0000:fffd9000       .debug$S                   0000000180000000     ucrt:api-ms-win-crt-string-l1-1-0.dll
 0000:fffd9000       .debug$S                   0000000180000000     ucrt:api-ms-win-crt-string-l1-1-0.dll
 0000:fffd9000       .debug$S                   0000000180000000     ucrt:api-ms-win-crt-string-l1-1-0.dll
 0000:fffd9000       .debug$S                   0000000180000000     ucrt:api-ms-win-crt-string-l1-1-0.dll
 0000:fffd9000       .debug$S                   0000000180000000     ucrt:api-ms-win-crt-string-l1-1-0.dll
 0000:fffd9000       .debug$S                   0000000180000000     ucrt:api-ms-win-crt-string-l1-1-0.dll
 0000:fffd9000       .debug$S                   0000000180000000     kernel32:KERNEL32.dll
 0000:fffd9000       .debug$S                   0000000180000000     kernel32:KERNEL32.dll
 0000:fffd9000       .debug$S                   0000000180000000     kernel32:KERNEL32.dll
 0000:fffd9000       .debug$S                   0000000180000000     kernel32:KERNEL32.dll
 0000:fffd9000       .debug$S                   0000000180000000     kernel32:KERNEL32.dll
 0000:fffd9000       .debug$S                   0000000180000000     kernel32:KERNEL32.dll
 0000:fffd9000       .debug$S                   0000000180000000     kernel32:KERNEL32.dll
 0000:fffd9000       .debug$S                   0000000180000000     kernel32:KERNEL32.dll
 0000:fffd9000       .debug$S                   0000000180000000     kernel32:KERNEL32.dll
 0000:fffd9000       .debug$S                   0000000180000000     kernel32:KERNEL32.dll
 0000:fffd9000       .debug$S                   0000000180000000     kernel32:KERNEL32.dll
 0000:fffd9000       .debug$S                   0000000180000000     kernel32:KERNEL32.dll
 0000:fffd9000       .debug$S                   0000000180000000     kernel32:KERNEL32.dll
 0000:fffd9000       .debug$S                   0000000180000000     kernel32:KERNEL32.dll
 0000:fffd9000       .debug$S                   0000000180000000     kernel32:KERNEL32.dll
 0000:fffd9000       .debug$S                   0000000180000000     kernel32:KERNEL32.dll
 0000:fffd9000       .debug$S                   0000000180000000     kernel32:KERNEL32.dll
 0000:fffd9000       .debug$S                   0000000180000000     kernel32:KERNEL32.dll
 0000:fffd9000       .debug$S                   0000000180000000     kernel32:KERNEL32.dll
 0000:fffd9000       .debug$S                   0000000180000000     kernel32:KERNEL32.dll
 0000:fffd9000       .debug$S                   0000000180000000     kernel32:KERNEL32.dll
 0000:fffd9000       .debug$S                   0000000180000000     kernel32:KERNEL32.dll
 0000:fffd9000       .debug$S                   0000000180000000     kernel32:KERNEL32.dll
 0000:fffd9000       .debug$S                   0000000180000000     kernel32:KERNEL32.dll
 0000:fffd9000       .debug$S                   0000000180000000     kernel32:KERNEL32.dll
 0000:fffd9000       .debug$S                   0000000180000000     kernel32:KERNEL32.dll
 0000:fffd9000       .debug$S                   0000000180000000     kernel32:KERNEL32.dll
 0000:fffd9000       .debug$S                   0000000180000000     kernel32:KERNEL32.dll
 0001:00001168       addRefToVerify             0000000180002168 f   libearlyretbase.obj
 0001:000011dc       agentThreadWrapper         00000001800021dc f   libearlyretbase.obj
 0001:000013b4       file_basename              00000001800023b4 f   libearlyretbase.obj
 0001:000019dc       startAgentThreadWrapper    00000001800029dc f   libearlyretbase.obj
 0001:00001edc       syncDebuggeeStatus         0000000180002edc f   libearlyretbase.obj
 0001:00002164       capture_previous_context   0000000180003164 f   MSVCRT:gs_report.obj
 0001:000021d8       ?__scrt_initialize_thread_safe_statics@@YAHXZ 00000001800031d8 f   MSVCRT:thread_safe_statics.obj
 0001:000022a8       ?__scrt_uninitialize_thread_safe_statics@@YAXXZ 00000001800032a8 f   MSVCRT:thread_safe_statics.obj
 0001:00002350       $$000000                   0000000180003350     MSVCRT:amdsecgs.obj
 0001:00002380       ?dllmain_crt_dispatch@@YAHQEAUHINSTANCE__@@KQEAX@Z 0000000180003380 f   MSVCRT:dll_dllmain.obj
 0001:000023d0       ?dllmain_crt_process_attach@@YAHQEAUHINSTANCE__@@QEAX@Z 00000001800033d0 f   MSVCRT:dll_dllmain.obj
 0001:000024e8       ?dllmain_crt_process_detach@@YAH_N@Z 00000001800034e8 f   MSVCRT:dll_dllmain.obj
 0001:0000256c       ?dllmain_dispatch@@YAHQEAUHINSTANCE__@@KQEAX@Z 000000018000356c f   MSVCRT:dll_dllmain.obj
 0001:00002f80       $$000000                   0000000180003f80     MSVCRT:guard_dispatch.obj
 0001:00002fa0       $$000000                   0000000180003fa0     MSVCRT:guard_xfg_dispatch.obj
 0001:00002fb6       ?fin$0@?0??dllmain_crt_process_attach@@YAHQEAUHINSTANCE__@@QEAX@Z@4HA 0000000180003fb6 f   MSVCRT:dll_dllmain.obj
 0001:00002fcd       ?fin$0@?0??dllmain_crt_process_detach@@YAH_N@Z@4HA 0000000180003fcd f   MSVCRT:dll_dllmain.obj
 0001:00002fe6       ?fin$1@?0??dllmain_crt_process_detach@@YAH_N@Z@4HA 0000000180003fe6 f   MSVCRT:dll_dllmain.obj
 0001:00002ffa       ?filt$0@?0??dllmain_dispatch@@YAHQEAUHINSTANCE__@@KQEAX@Z@4HA 0000000180003ffa f   MSVCRT:dll_dllmain.obj
 0001:00003030       __scrt_is_nonwritable_in_current_image$filt$0 0000000180004030 f   MSVCRT:utility.obj
 0002:000001e8       ?__scrt_initialize_tss_var@@3P6AHXZEA 00000001800051e8     MSVCRT:thread_safe_statics.obj
 0002:00000310       ?opcLengths@@3QBEB         0000000180005310     libearlyretbase.obj
 0002:00002050       GS_ExceptionPointers       0000000180007050     MSVCRT:gs_report.obj
 0002:00002728       $unwind$fprintf            0000000180007728     libearlyretbase.obj
 0002:00002734       $unwind$printf             0000000180007734     libearlyretbase.obj
 0002:00002740       $unwind$?NewObject@JNIEnv_@@QEAAPEAV_jobject@@PEAV_jclass@@PEAU_jmethodID@@ZZ 0000000180007740     libearlyretbase.obj
 0002:00002740       $unwind$nsk_lcomplain      0000000180007740     libearlyretbase.obj
 0002:00002740       $unwind$nsk_ldisplay       0000000180007740     libearlyretbase.obj
 0002:00002748       $unwind$nsk_lvdisplay      0000000180007748     libearlyretbase.obj
 0002:00002748       $unwind$_RTC_Initialize    0000000180007748     MSVCRT:initsect.obj
 0002:00002748       $unwind$_RTC_Terminate     0000000180007748     MSVCRT:initsect.obj
 0002:00002748       $unwind$?__scrt_initialize_thread_safe_statics@@YAHXZ 0000000180007748     MSVCRT:thread_safe_statics.obj
 0002:00002754       $unwind$nsk_lvcomplain     0000000180007754     libearlyretbase.obj
 0002:0000276c       $unwind$nsk_ltrace         000000018000776c     libearlyretbase.obj
 0002:0000276c       $unwind$__report_gsfailure 000000018000776c     MSVCRT:gs_report.obj
 0002:00002774       $unwind$Agent_Initialize   0000000180007774     libearlyretbase.obj
 0002:00002774       $unwind$Java_nsk_jvmti_unit_ForceEarlyReturn_earlyretbase_check 0000000180007774     libearlyretbase.obj
 0002:00002774       $unwind$Java_nsk_jvmti_unit_ForceEarlyReturn_earlyretbase_resThread 0000000180007774     libearlyretbase.obj
 0002:00002774       $unwind$nsk_lvtrace        0000000180007774     libearlyretbase.obj
 0002:00002774       $unwind$__raise_securityfailure 0000000180007774     MSVCRT:gs_report.obj
 0002:00002774       $unwind$__scrt_initialize_crt 0000000180007774     MSVCRT:utility.obj
 0002:00002774       $unwind$__scrt_initialize_onexit_tables 0000000180007774     MSVCRT:utility.obj
 0002:00002774       $unwind$__scrt_release_startup_lock 0000000180007774     MSVCRT:utility.obj
 0002:00002774       $unwind$__scrt_uninitialize_crt 0000000180007774     MSVCRT:utility.obj
 0002:00002774       $unwind$_onexit            0000000180007774     MSVCRT:utility.obj
 0002:0000277c       $unwind$nsk_lverify        000000018000777c     libearlyretbase.obj
 0002:0000278c       $unwind$nsk_vprintf        000000018000778c     libearlyretbase.obj
 0002:0000279c       $unwind$nsk_printf         000000018000779c     libearlyretbase.obj
 0002:000027a4       $unwind$?nsk_jni_lverify@@YAHHPEAUJNIEnv_@@HQEBDH1ZZ 00000001800077a4     libearlyretbase.obj
 0002:000027b8       $unwind$?nsk_jni_check_exception@@YAHPEAUJNIEnv_@@QEBDH@Z 00000001800077b8     libearlyretbase.obj
 0002:000027d4       $unwind$FramePop           00000001800077d4     libearlyretbase.obj
 0002:000027d4       $unwind$Java_nsk_jvmti_unit_FollowReferences_FollowRefObjects_resetTags 00000001800077d4     libearlyretbase.obj
 0002:000027d4       $unwind$MethodExit         00000001800077d4     libearlyretbase.obj
 0002:000027d4       $unwind$addRefToVerify     00000001800077d4     libearlyretbase.obj
 0002:000027d4       $unwind$nsk_jvmti_resetAgentData 00000001800077d4     libearlyretbase.obj
 0002:000027d4       $unwind$__scrt_initialize_default_local_stdio_options 00000001800077d4     MSVCRT:default_local_stdio_options.obj
 0002:000027d4       $unwind$?dllmain_crt_dispatch@@YAHQEAUHINSTANCE__@@KQEAX@Z 00000001800077d4     MSVCRT:dll_dllmain.obj
 0002:000027d4       $unwind$DllMain            00000001800077d4     MSVCRT:dll_dllmain_stub.obj
 0002:000027d4       $unwind$__GSHandlerCheck   00000001800077d4     MSVCRT:gshandler.obj
 0002:000027d4       $unwind$?__scrt_uninitialize_thread_safe_statics@@YAXXZ 00000001800077d4     MSVCRT:thread_safe_statics.obj
 0002:000027d4       $unwind$__scrt_acquire_startup_lock 00000001800077d4     MSVCRT:utility.obj
 0002:000027d4       $unwind$__scrt_dllmain_after_initialize_c 00000001800077d4     MSVCRT:utility.obj
 0002:000027d4       $unwind$__scrt_dllmain_before_initialize_c 00000001800077d4     MSVCRT:utility.obj
 0002:000027d4       $unwind$__scrt_dllmain_crt_thread_attach 00000001800077d4     MSVCRT:utility.obj
 0002:000027d4       $unwind$__scrt_dllmain_crt_thread_detach 00000001800077d4     MSVCRT:utility.obj
 0002:000027d4       $unwind$__scrt_dllmain_uninitialize_c 00000001800077d4     MSVCRT:utility.obj
 0002:000027d4       $unwind$__scrt_dllmain_uninitialize_critical 00000001800077d4     MSVCRT:utility.obj
 0002:000027d4       $unwind$atexit             00000001800077d4     MSVCRT:utility.obj
 0002:000027dc       $unwind$nsk_jvmti_lverify  00000001800077dc     libearlyretbase.obj
 0002:000027f0       $unwind$suspendThreadAtMethod 00000001800077f0     libearlyretbase.obj
 0002:00002808       $unwind$exitOnError        0000000180007808     libearlyretbase.obj
 0002:00002818       $unwind$Java_nsk_share_jvmti_ArgumentHandler_getAgentOptionsString 0000000180007818     libearlyretbase.obj
 0002:0000282c       $unwind$Java_nsk_jvmti_unit_FollowReferences_FollowRefObjects_getTag 000000018000782c     libearlyretbase.obj
 0002:0000282c       $unwind$Java_nsk_share_jvmti_DebugeeClass_checkStatus 000000018000782c     libearlyretbase.obj
 0002:0000282c       $unwind$agentThreadWrapper 000000018000782c     libearlyretbase.obj
 0002:0000283c       $unwind$startAgentThreadWrapper 000000018000783c     libearlyretbase.obj
 0002:00002858       $unwind$syncDebuggeeStatus 0000000180007858     libearlyretbase.obj
 0002:00002858       $unwind$__scrt_dllmain_exception_filter 0000000180007858     MSVCRT:utility.obj
 0002:0000286c       $unwind$Java_nsk_share_jvmti_DebugeeClass_resetAgentData 000000018000786c     libearlyretbase.obj
 0002:00002874       $unwind$MA_checkStatus     0000000180007874     libearlyretbase.obj
 0002:00002888       $unwind$Java_nsk_jvmti_unit_FollowReferences_FollowRefObjects_setTag 0000000180007888     libearlyretbase.obj
 0002:000028a0       $unwind$Java_nsk_jvmti_unit_FollowReferences_FollowRefObjects_addRefToVerify 00000001800078a0     libearlyretbase.obj
 0002:000028bc       $unwind$Java_nsk_jvmti_unit_ForceEarlyReturn_earlyretbase_doForceEarlyReturn 00000001800078bc     libearlyretbase.obj
 0002:000028bc       $unwind$Java_nsk_jvmti_unit_ForceEarlyReturn_earlyretbase_suspThread 00000001800078bc     libearlyretbase.obj
 0002:000028bc       $unwind$_DllMainCRTStartup 00000001800078bc     MSVCRT:dll_dllmain.obj
 0002:000028cc       $unwind$capture_previous_context 00000001800078cc     MSVCRT:gs_report.obj
 0002:000028d8       $unwind$__GSHandlerCheckCommon 00000001800078d8     MSVCRT:gshandler.obj
 0002:000028e0       $xdatasym                  00000001800078e0     MSVCRT:amdsecgs.obj
 0002:000028e4       $unwind$?dllmain_crt_process_attach@@YAHQEAUHINSTANCE__@@QEAX@Z 00000001800078e4     MSVCRT:dll_dllmain.obj
 0002:00002920       $unwind$?fin$0@?0??dllmain_crt_process_attach@@YAHQEAUHINSTANCE__@@QEAX@Z@4HA 0000000180007920     MSVCRT:dll_dllmain.obj
 0002:00002920       $unwind$?fin$0@?0??dllmain_crt_process_detach@@YAH_N@Z@4HA 0000000180007920     MSVCRT:dll_dllmain.obj
 0002:00002920       $unwind$?fin$1@?0??dllmain_crt_process_detach@@YAH_N@Z@4HA 0000000180007920     MSVCRT:dll_dllmain.obj
 0002:00002928       $unwind$?dllmain_crt_process_detach@@YAH_N@Z 0000000180007928     MSVCRT:dll_dllmain.obj
 0002:0000297c       $unwind$?dllmain_dispatch@@YAHQEAUHINSTANCE__@@KQEAX@Z 000000018000797c     MSVCRT:dll_dllmain.obj
 0002:000029a4       $unwind$?filt$0@?0??dllmain_dispatch@@YAHQEAUHINSTANCE__@@KQEAX@Z@4HA 00000001800079a4     MSVCRT:dll_dllmain.obj
 0002:000029ac       $unwind$__scrt_is_nonwritable_in_current_image 00000001800079ac     MSVCRT:utility.obj
 0002:000029cc       $unwind$__scrt_is_nonwritable_in_current_image$filt$0 00000001800079cc     MSVCRT:utility.obj
 0002:000029d4       $unwind$__scrt_fastfail    00000001800079d4     MSVCRT:utility_desktop.obj
 0002:000029e4       $unwind$__security_init_cookie 00000001800079e4     MSVCRT:gs_support.obj
 0002:000029f0       $unwind$__isa_available_init 00000001800079f0     MSVCRT:cpu_disp.obj
 0002:00002a00       $xdatasym                  0000000180007a00     MSVCRT:guard_dispatch.obj
 0002:00002a08       $xdatasym                  0000000180007a08     MSVCRT:guard_xfg_dispatch.obj
 0002:00002a10       .edata                     0000000180007a10     earlyretbase.exp
 0002:00002a38       rgpv                       0000000180007a38     earlyretbase.exp
 0002:00002a80       rgszName                   0000000180007a80     earlyretbase.exp
 0002:00002ac8       rgwOrd                     0000000180007ac8     earlyretbase.exp
 0002:00002aec       szName                     0000000180007aec     earlyretbase.exp
 0002:00002afd       $N00001                    0000000180007afd     earlyretbase.exp
 0002:00002b0c       $N00002                    0000000180007b0c     earlyretbase.exp
 0002:00002b19       $N00003                    0000000180007b19     earlyretbase.exp
 0002:00002b5e       $N00004                    0000000180007b5e     earlyretbase.exp
 0002:00002b9b       $N00005                    0000000180007b9b     earlyretbase.exp
 0002:00002be3       $N00006                    0000000180007be3     earlyretbase.exp
 0002:00002c23       $N00007                    0000000180007c23     earlyretbase.exp
 0002:00002c60       $N00008                    0000000180007c60     earlyretbase.exp
 0002:00002c98       $N00009                    0000000180007c98     earlyretbase.exp
 0002:00002cdd       $N00010                    0000000180007cdd     earlyretbase.exp
 0002:00002d19       $N00011                    0000000180007d19     earlyretbase.exp
 0002:00002d56       $N00012                    0000000180007d56     earlyretbase.exp
 0002:00002d91       $N00013                    0000000180007d91     earlyretbase.exp
 0002:00002dbf       $N00014                    0000000180007dbf     earlyretbase.exp
 0002:00002df0       $N00015                    0000000180007df0     earlyretbase.exp
 0002:00002e1f       $N00016                    0000000180007e1f     earlyretbase.exp
 0002:00002e4e       $N00017                    0000000180007e4e     earlyretbase.exp
 0002:00002e83       $N00018                    0000000180007e83     earlyretbase.exp
 0002:0000329a       .idata$6                   000000018000829a     kernel32:KERNEL32.dll
 0002:000032fe       .idata$6                   00000001800082fe     vcruntime:VCRUNTIME140.dll
 0002:00003460       .idata$6                   0000000180008460     ucrt:api-ms-win-crt-runtime-l1-1-0.dll
 0002:00003482       .idata$6                   0000000180008482     ucrt:api-ms-win-crt-stdio-l1-1-0.dll
 0002:000034a2       .idata$6                   00000001800084a2     ucrt:api-ms-win-crt-string-l1-1-0.dll
 0003:00000000       ?codeAttributeName@@3PEBDEB 0000000180009000     libearlyretbase.obj
 0003:00000008       ?lineNumberAttributeName@@3PEBDEB 0000000180009008     libearlyretbase.obj
 0003:00000010       ?localVarAttributeName@@3PEBDEB 0000000180009010     libearlyretbase.obj
 0003:00000018       ?localVarTypeAttributeName@@3PEBDEB 0000000180009018     libearlyretbase.obj
 0003:00000020       ?stackMapAttributeName@@3PEBDEB 0000000180009020     libearlyretbase.obj
 0003:00000028       ?callBytes@@3PAEA          0000000180009028     libearlyretbase.obj
 0003:0000002c       ?allocBytes@@3PAEA         000000018000902c     libearlyretbase.obj
 0003:00000030       sig_exp                    0000000180009030     libearlyretbase.obj
 0003:00000038       name_exp                   0000000180009038     libearlyretbase.obj
 0003:0001aae4       redefineAttempted          0000000180023ae4     libearlyretbase.obj
 0003:0001aae8       nsk_context                0000000180023ae8     libearlyretbase.obj
 0003:0001aaf4       redefineSucceed            0000000180023af4     libearlyretbase.obj
 0003:0001aaf8       agentFailed                0000000180023af8     libearlyretbase.obj
 0003:0001aafc       currentAgentStatus         0000000180023afc     libearlyretbase.obj
 0003:0001ab00       context                    0000000180023b00     libearlyretbase.obj
 0003:0001abb8       agentThread                0000000180023bb8     libearlyretbase.obj
 0003:0001abc0       agentThreadProc            0000000180023bc0     libearlyretbase.obj
 0003:0001abc8       agentThreadArg             0000000180023bc8     libearlyretbase.obj
 0003:0001abd0       agent_data                 0000000180023bd0     libearlyretbase.obj
 0003:0001abe0       jvmti_env                  0000000180023be0     libearlyretbase.obj
 0003:0001abe8       jvm                        0000000180023be8     libearlyretbase.obj
 0003:0001abf0       jni_env                    0000000180023bf0     libearlyretbase.obj
 0003:0001abf8       checkStatus_func           0000000180023bf8     libearlyretbase.obj
 0003:0001ac00       ?codeAttributeIndex@@3GA   0000000180023c00     libearlyretbase.obj
 0003:0001ac04       ?lineNumberAttributeIndex@@3GA 0000000180023c04     libearlyretbase.obj
 0003:0001ac08       ?localVarAttributeIndex@@3GA 0000000180023c08     libearlyretbase.obj
 0003:0001ac0c       ?localVarTypeAttributeIndex@@3GA 0000000180023c0c     libearlyretbase.obj
 0003:0001ac10       ?stackMapAttributeIndex@@3GA 0000000180023c10     libearlyretbase.obj
 0003:0001ac14       ?stackFrameOffset@@3GA     0000000180023c14     libearlyretbase.obj
 0003:0001ac18       ?mode@@3HA                 0000000180023c18     libearlyretbase.obj
 0003:0001ac1c       ?constantPoolSize@@3GA     0000000180023c1c     libearlyretbase.obj
 0003:0001ac20       ?orig@@3PEBEEB             0000000180023c20     libearlyretbase.obj
 0003:0001ac28       ?gen@@3PEAEEA              0000000180023c28     libearlyretbase.obj
 0003:0001ac30       ?inputPos@@3PEAEEA         0000000180023c30     libearlyretbase.obj
 0003:0001ac38       ?endPos@@3PEBEEB           0000000180023c38     libearlyretbase.obj
 0003:0001ac40       ?genPos@@3PEAEEA           0000000180023c40     libearlyretbase.obj
 0003:0001ac48       ?markPos@@3PEAEEA          0000000180023c48     libearlyretbase.obj
 0003:0001ac50       ?constantPool@@3PEAPEADEA  0000000180023c50     libearlyretbase.obj
 0003:0001ac58       ?constantPoolCount@@3GA    0000000180023c58     libearlyretbase.obj
 0003:0001ac5c       ?zeroBytes@@3PAEA          0000000180023c5c     libearlyretbase.obj
 0003:0001ac60       ?codeLength@@3IA           0000000180023c60     libearlyretbase.obj
 0003:0001ac64       meth_exit_exp_events       0000000180023c64     libearlyretbase.obj
 0003:0001ac68       ?map@@3PEAIEA              0000000180023c68     libearlyretbase.obj
 0003:0001ac70       ?widening@@3PEACEA         0000000180023c70     libearlyretbase.obj
 0003:0001ac78       jvmti                      0000000180023c78     libearlyretbase.obj
 0003:0001ac80       caps                       0000000180023c80     libearlyretbase.obj
 0003:0001ac90       callbacks                  0000000180023c90     libearlyretbase.obj
 0003:0001adc8       pop_frame_exp_events       0000000180023dc8     libearlyretbase.obj
 0003:0001adcc       meth_exit_gen_events       0000000180023dcc     libearlyretbase.obj
 0003:0001add0       pop_frame_gen_events       0000000180023dd0     libearlyretbase.obj
 0003:0001add4       errCode                    0000000180023dd4     libearlyretbase.obj
 0003:0001add8       midActiveMethod            0000000180023dd8     libearlyretbase.obj
 0003:0001adf0       GS_ExceptionRecord         0000000180023df0     MSVCRT:gs_report.obj
 0003:0001ae90       GS_ContextRecord           0000000180023e90     MSVCRT:gs_report.obj
 0003:0001b360       ?g_tss_cv@@3U_RTL_CONDITION_VARIABLE@@A 0000000180024360     MSVCRT:thread_safe_statics.obj
 0003:0001b368       ?g_tss_event@@3PEAXEA      0000000180024368     MSVCRT:thread_safe_statics.obj
 0003:0001b370       ?g_tss_mutex@@3U_RTL_CRITICAL_SECTION@@A 0000000180024370     MSVCRT:thread_safe_statics.obj
 0003:0001b398       ?g_sleep_condition_variable_cs@@3P6AHPEAU_RTL_CONDITION_VARIABLE@@PEAU_RTL_CRITICAL_SECTION@@K@ZEA 0000000180024398     MSVCRT:thread_safe_statics.obj
 0003:0001b3a0       ?g_wake_all_condition_variable@@3P6AXPEAU_RTL_CONDITION_VARIABLE@@@ZEA 00000001800243a0     MSVCRT:thread_safe_statics.obj
 0003:0001b3ac       ?__proc_attached@@3HA      00000001800243ac     MSVCRT:dll_dllmain.obj
 0003:0001b3c0       ?is_initialized_as_dll@@3_NA 00000001800243c0     MSVCRT:utility.obj
 0003:0001b3c1       ?module_local_atexit_table_initialized@@3_NA 00000001800243c1     MSVCRT:utility.obj
 0003:0001b3c8       ?module_local_atexit_table@@3U_onexit_table_t@@A 00000001800243c8     MSVCRT:utility.obj
 0003:0001b3e0       ?module_local_at_quick_exit_table@@3U_onexit_table_t@@A 00000001800243e0     MSVCRT:utility.obj
